S01900006F70656E626C745F73746D3332663734362E73726563F8
S3150800000050140020055F0008395F00083D5F0008AE
S31508000010415F0008455F0008495F000800000000CE
S315080000200000000000000000000000004D5F00080E
S31508000030515F000800000000555F000871110008B4
S31508000040595F00085D5F0008615F0008655F00088A
S31508000050695F00086D5F0008715F0008755F00083A
S31508000060795F00087D5F0008815F0008855F0008EA
S31508000070895F00088D5F0008915F0008955F00089A
S31508000080995F00089D5F0008A15F0008A55F00084A
S31508000090A95F0008AD5F0008B15F0008B55F0008FA
S315080000A0B95F0008BD5F0008C15F0008C55F0008AA
S315080000B0C95F0008CD5F0008D15F0008D55F00085A
S315080000C0D95F0008DD5F0008E15F0008E55F00080A
S315080000D0E95F0008ED5F0008F15F0008F55F0008BA
S315080000E0F95F0008FD5F0008016000080560000868
S315080000F0096000080D600008116000081560000816
S31508000100196000081D6000082160000825600008C5
S31508000110296000082D600008316000083560000875
S31508000120396000083D600008416000084560000825
S31508000130496000084D6000085160000855600008D5
S31508000140596000085D600008616000086560000885
S31508000150696000086D600008716000087560000835
S31508000160796000087D6000088160000885600008E5
S31508000170896000088D600008916000080000000092
S3150800018095600008996000089D600008A160000855
S31508000190A5600008A9600008AD600008B160000805
S315080001A0B5600008B9600008BD600008C1600008B5
S315080001B0C5600008C9600008CD600008D160000865
S315080001C0D5600008D96000080EB418B50400089870
S315080001D0012817D1A06B30F48030A063E168DFF8FE
S315080001E030090140E160E06830F44010E0600F98A3
S315080001F0012803D1E06850F48010E060200000F088
S315080002004BFF0AE0E06850F04000E060200000F094
S3150800021043FFA16B51F48031A1630699012907D1E7
S31508000220A16851F00601A160A16851F02001A16002
S31508000230C0B212BC5DF810FB1300DBB2022B52D120
S31508000240DFF8D0288A1ADFF8D0389A4201D20F216F
S315080002504FE0DFF8C8288A1ADFF8C4389A4201D274
S315080002600E2146E0DFF8BC288A1ADFF8BC389A4225
S3150800027001D20D213DE0DFF8B4288A1ADFF8B0383C
S315080002809A4201D20C2134E0DFF8A8288A1ADFF84E
S31508000290A8389A4201D20B212BE0DFF8A0288A1A47
S315080002A0DFF89C389A4201D20A2122E0DFF8942826
S315080002B08A1ADFF894389A4201D2092119E0DFF840
S315080002C08C288A1ADFF888389A4201D2082110E069
S315080002D0DFF88028891ADFF88028914201D20721A1
S315080002E007E0062105E0D2B2002A01D1092100E083
S315080002F00921C26832F47052C260C268890211F4D8
S3150800030070511143C16000207047816851F00101A6
S315080003108160002070478168490849008160002093
S31508000320704780B5C26832F0C042C2600A00D2B2D5
S31508000330012A08D1C16851F00051C160322000F08D
S31508000340D1FE002002BDC9B2002904D1C16851F00E
S315080003508041C160F2E70120F4E70EB478B50400E5
S3150800036000252600002005E0002104EB8002C2F8E3
S315080003700411401C0F28F7D30F98002814D116F53E
S315080003800060406850F0020016F500614860A06BF6
S3150800039030F40010A063206850F040002060206808
S315080003A050F08000206003E0A06B50F40010A063BA
S315080003B0002016F56061086016F50060006816F5FD
S315080003C0006108600A9801280CD10798002804D112
S315080003D00021200000F0E5F818E00121200000F0D7
S315080003E0E0F813E00A9803280CD10798002804D1EE
S315080003F00021200000F0D5F808E00121200000F0D7
S31508000400D0F803E00321200000F0CBF810212000EB
S3150800041000F0A7F8002800D00125200000F0B2F867
S31508000420002800D00125002016F50061086100208B
S3150800043016F500614861002016F50061C8610020C4
S315080004401BE0002116EB401212F51062116006E05F
S315080004505FF0904116EB401212F51062116016EB30
S31508000460401111F5106100220A6116EB401111F5D1
S3150800047010614FF67F328A60401C0599884210D277
S3150800048016EB401111F5106109680029D9D5002825
S31508000490DED15FF0006116EB401212F510621160B2
S315080004A0DDE700201BE0002116EB401212F5306252
S315080004B0116006E05FF0904116EB401212F53062CB
S315080004C0116016EB401111F5306100220A6116EB36
S315080004D0401111F530614FF67F328A60401C05994C
S315080004E0884210D216EB401111F5306109680029CF
S315080004F0D9D50028DED15FF0006116EB401212F55F
S3150800050030621160DDE716F50060006930F480702E
S3150800051016F5006630610020A0617FF080406061BA
S315080005200898002803D1A06950F01000A061A169BD
S31508000530DFF8980B0143A1610B98002803D0A06946
S3150800054050F00800A0610F98012805D1A06940F075
S31508000550804050F00400A0612800C0B272BC5DF86B
S3150800056010FB0022890151F020010161521CDFF8BD
S31508000570601B8A4204D201698906F7D400207047B5
S315080005800320FCE7002110220261491CDFF8402BFA
S31508000590914204D20269D206F7D40020704703209C
S315080005A0FCE710F500621268C9B2114310F5006045
S315080005B001600020704710F50060806810F00600A2
S315080005C0002801D1002006E0022801D0062801D122
S315080005D0022000E00F20C0B2704730B40A784B788A
S315080005E0012B2BD110F50063DB6901240D7815F07A
S315080005F00F05AC40A4B2234310F50064E36110EB89
S31508000600421313F510631B681B0440D410EB421306
S3150800061013F510631B688C686405640DC97854EA81
S31508000620814454EA825444F0805454F400442343E9
S3150800063010EB421010F51060036028E010F5006317
S31508000640DB6901240D7815F00F05AC4053EA044325
S3150800065010F50064E36110EB421313F530631B6871
S315080006601B0414D410EB421313F530631B688C6813
S315080006706405640DC97854EA814444F0805454F4FE
S315080006800044234310EB421010F53060036000204D
S3150800069030BC704730B40A784B78012B47D110EB41
S315080006A0421313F510631B68002B17D510EB421382
S315080006B013F510631B6853F0006310EB421414F52E
S315080006C01064236010EB421313F510631B6853F094
S315080006D0804310EB421414F510642360012310F5CF
S315080006E00064E46B0D7815F00F0513FA05F5ADB245
S315080006F0AC4310F50065EC6310F50064E46909780D
S3150800070011F00F018B409BB234EA030310F5006128
S31508000710CB6110EB421111F510610B68DFF8B419C3
S315080007200B4010EB421010F51060036045E010EB2B
S31508000730421313F530631B68002B17D510EB4213D1
S3150800074013F530631B6853F0006310EB421414F57D
S315080007503064236010EB421313F530631B6853F0C3
S31508000760804310EB421414F530642360012310F51E
S315080007700064E46B0D7815F00F0513FA05F534EAF5
S31508000780054410F50065EC6310F50064E469097822
S3150800079011F00F018B4034EA034410F50061CC6177
S315080007A010EB421111F530610B68DFF82C190B407C
S315080007B010EB421010F530600360002030BC704723
S315080007C0F8B504000D784B78012B40F005814B698C
S315080007D0002B24D114EB451313F5106314EB4516BF
S315080007E016F5106636696FF3DC461E6114EB451381
S315080007F013F5106314EB451616F51066366956F4AC
S3150800080000261E6114EB451313F5106314EB451609
S3150800081016F510663669F60CF6041E615AE014EBF6
S31508000820451313F5106314EB451616F5106636696D
S31508000830F60CF6041E6114EB451313F5106314EB5E
S31508000840451616F5106636696FF3DC461E6114EB1D
S31508000850451616F5106614EB451313F510631F6954
S31508000860D1F814C08B6813EB0C0CBCF1010C8B6827
S31508000870BCFBF3F3DFF864C81CEAC34C5CEA070761
S31508000880376114EB451313F5106314EB451616F58B
S31508000890106636694F697F037F0B3E431E61CB782E
S315080008A0012B17D114EB451313F5106314EB4516FA
S315080008B016F51066366936F0C0461E6114EB451308
S315080008C013F5106314EB451616F51066366956F0DF
S315080008D000561E611300DBB2012B36D108690028C9
S315080008E005D014EB451010F510600A694261C87806
S315080008F001281DD114F500608068C0050CD414EBDE
S31508000900451010F51060006850F0005014EB4511C2
S3150800091011F5106108600BE014EB451010F5106036
S31508000920006850F0805014EB451111F5106108600D
S3150800093014EB451010F51060006850F0044014EBF5
S31508000940451414F510642060DFE014EB451313F525
S3150800095010631B6853F0044314EB451616F510662E
S315080009603360CB78012B10D04869002800F0CD8081
S3150800097014F50060406B0122097811F00F018A40D6
S31508000980104314F500646063BFE014F500639B68C8
S31508000990DB050CD414EB451313F510631B6853F0F1
S315080009A0005314EB451414F5106423600BE014EBA4
S315080009B0451313F510631B6853F0805314EB451465
S315080009C014F510642360D2B200924B699BB20A7880
S315080009D0C96800F0B1F998E014EB451010F53060DD
S315080009E014EB451313F530631B69DB0CDB04036159
S315080009F014EB451010F5306014EB451313F530630E
S31508000A001B696FF3DC430361486900281AD114EBAC
S31508000A10451010F5306014EB451313F530631B6968
S31508000A208E687603760B3343036114EB451010F595
S31508000A30306014EB451313F530631B6953F4002338
S31508000A40036129E04B698868C3185B1E8868B3FB95
S31508000A50F0F014EB451313F5306314EB451616F551
S31508000A60306636690700BFB2DFF870C61CEAC74CA5
S31508000A705CEA06061E6114EB451313F5306314EBA6
S31508000A80451616F5306636698F6880B200FB07F0A2
S31508000A904003400B30431861D2B2012A08D1C86816
S31508000AA0002805D014EB451010F53060CA6842617D
S31508000AB0C87801281DD114F500608068C0050CD4DB
S31508000AC014EB451010F53060006850F0005014EB38
S31508000AD0451111F5306108600BE014EB451010F56F
S31508000AE03060006850F0805014EB451111F5306104
S31508000AF0086014EB451010F53060006850F00440AB
S31508000B0014EB451414F5306420600020F2BD000093
S31508000B10BFFFBDFFC0ACD80000350C00C0E1E40043
S31508000B2040420F000024F400804F12008073060133
S31508000B3020D61300A0491A0160E31600002D3101E2
S31508000B4040771B0040A44C01C091210000366E017D
S31508000B502075380020ABA601E09C410070B40B005C
S31508000B601C785978012940F095805969002924D1C3
S31508000B7010EB441111F5106110EB441515F51065CD
S31508000B802D696FF3DC450D6110EB441111F5106109
S31508000B9010EB441515F510652D6955F400250D6102
S31508000BA010EB441111F5106110EB441515F510659D
S31508000BB02D69ED0CED040D6137E010EB441111F5CC
S31508000BC0106110EB441515F510652D69ED0CED0453
S31508000BD00D6110EB441111F5106110EB441515F574
S31508000BE010652D696FF3DC450D6199685D69A94249
S31508000BF001D29968596110EB441111F5106110EB97
S31508000C00441515F510652D6955F400250D6110EB91
S31508000C10441111F5106110EB441515F510652D6991
S31508000C205E697603760B35430D61D2B2012A15D17A
S31508000C301969002905D010EB441111F510611A69DC
S31508000C404A6110EB441111F51061096851F004412D
S31508000C5010EB441010F5106001606AE010EB4411C7
S31508000C6011F51061096851F0044110EB441212F5B0
S31508000C7010621160596900295BD010F50061496B53
S31508000C8001221B7813F00F039A40114310F50060F8
S31508000C9041634EE010EB441111F5306110EB441539
S31508000CA015F530652D69ED0CED040D6110EB441159
S31508000CB011F5306110EB441515F530652D696FF3A4
S31508000CC0DC450D615969002901D09968596110EB15
S31508000CD0441111F5306110EB441515F530652D6991
S31508000CE055F400250D6110EB441111F5306110EB38
S31508000CF0441515F530652D699E687603760B3543E0
S31508000D000D61D2B2012A08D1D968002905D010EBA5
S31508000D10441111F53061DA684A6110EB441111F596
S31508000D203061096851F0044110EB441010F5306049
S31508000D300160002070BC7047F0B4049CE4B2002C3B
S31508000D4013D19BB2DB1C9B0800250CE00C0026681F
S31508000D501700FFB24FF4805404FB070717F58057B6
S31508000D603E60091D6D1C9D42F0D30020F0BC704703
S31508000D7030B492B2D21C9208002306E010F58054D3
S31508000D8024680D002C60091D5B1C9342F6D30800ED
S31508000D9030BC7047020008784978012921D112EB46
S31508000DA0401111F51061096800290DD400280BD0EF
S31508000DB012EB401111F51061096831F0804112EB10
S31508000DC0401313F51063196012EB401111F5106109
S31508000DD0096851F4001112EB401212F51062116005
S31508000DE020E012EB401111F53061096800290DD495
S31508000DF000280BD012EB401111F53061096831F06B
S31508000E00804112EB401313F53063196012EB401161
S31508000E1011F53061096851F4001112EB401212F510
S31508000E20306211600020704710B40A784B78012BA5
S31508000E301ED110EB421313F510631B6833F400132D
S31508000E4010EB421414F510642360CB78032B02D000
S31508000E50C97802292AD110EB421111F510610968E7
S31508000E6051F0805110EB421010F5106001601DE042
S31508000E7010EB421313F530631B6833F4001310EBC1
S31508000E80421414F530642360CB78032B02D0C9785A
S31508000E9002290BD110EB421111F53061096851F0A6
S31508000EA0805110EB421010F530600160002010BC34
S31508000EB0704710B50400200000210CE04FF67F3281
S31508000EC010EB411313F510639A6010EB411313F5F9
S31508000ED030639A60491C0F29F0D3002110F500628F
S31508000EE01161002110F500625161002110F50060C2
S31508000EF0C1612000FFF746FB0100C9B2002901D0F5
S31508000F00C0B20AE010212000FFF72BFB0100C9B28E
S31508000F10002901D0C0B200E0C0B210BD10F50062D1
S31508000F20126832F4FE6210F500631A6010F500626A
S31508000F301268C9B2090111F4FE61114310F5006087
S31508000F4001600020704780B510F50061496831F0EE
S31508000F50020110F500604160032000F0C3F800208C
S31508000F6002BD80B510F50061496851F0020110F51F
S31508000F7000604160032000F0B5F8002002BD0100C2
S31508000F804869896908407047010011F50060806961
S31508000F9011F50061C9690840000C7047010011F598
S31508000FA00060806911F50061C969084080B2704720
S31508000FB00200C9B212EB411010F53060806812F5D4
S31508000FC0006251690840704710B410F50062126952
S31508000FD010F500635B6B11F00F04E340DB0113F0BF
S31508000FE080031A43C9B210EB411010F510608068EF
S31508000FF0104010BC7047406910F00100704710F5AA
S3150800100010610968C90AC90210F51062116010F565
S315080010100061496851F4807110F500604160002054
S31508001020704710B40300006CDFF8B440A04206D342
S3150800103013F530600068002801D500202AE000205A
S3150800104013F53064206113F53060006950F4002010
S3150800105013F53064206113F53060006950F018000C
S3150800106013F53064206113F53060006950F0C04014
S3150800107013F530642061C9B201290AD113F530602D
S31508001080426113F53060006850F0802013F5306334
S315080010901860002010BC70470021491C0C4A914278
S315080010A00FD20369002BF8D50021036953F0010319
S315080010B00361491C914206D20369DB07F9D4002073
S315080010C070470320FCE70320FAE7000000383C805D
S315080010D0410D0300007833EC0078F3EF0000F81FA9
S315080010E00B30544F38B5040000F03EF8050014F1F3
S315080010F0010F02D004480078241800F035F8401B88
S31508001100A042FAD331BD00BFBD00002080B500F073
S315080011100DF810481049086000201049086005209D
S315080011200F49086000200F49086001BD00200C49DE
S31508001130086070470A480068C00303D50948016873
S31508001140491C0160704780B5FFF7F4FF0548006841
S3150800115002BD0000BF4B030014E000E018E000E009
S3150800116010E000E03810002080B5FFF7ECFF02BD64
S31508001170704730B4002513E050F8042BD30744BF5A
S31508001180A9F101039A18091F042942F8045BFAD247
S3150800119013468C0744BF15809B1CC90748BF1D70A2
S315080011A050F8041B0029E7D130BC704738B58AB01F
S315080011B00400002C01D10120B6E0256894F8BD038F
S315080011C0002805D1002084F8BC03200000F054FE56
S315080011D0032084F8BD03E86BC00501D40020206114
S315080011E02068FFF798F8211D83B06846342200F07E
S315080011F045FE0EBC2068FEF7E7FF002804D0022053
S3150800120084F8BD0301208FE000212068FFF789F8E4
S31508001210002130E01C200A00D2B2424322440123B6
S3150800122082F83D300A00D2B24243224482F83C108A
S315080012300A00D2B2424322440B00DBB2A2F8423083
S315080012400A00D2B242432244002382F83F300A0001
S31508001250D2B242432244002353640A00D2B2424324
S315080012602244002393640A00D2B200FB02F0204411
S3150800127000220265491C0800C0B262689042C9D3C0
S3150800128000212BE01C200A00D2B24243224400234C
S3150800129082F8FD310A00D2B24243224482F8FC1198
S315080012A00A00D2B242432244002382F8FF310A00E0
S315080012B0D2B2424322440023C2F804320A00D2B210
S315080012C0424322440023C2F808320A00D2B200FB85
S315080012D002F020440022C0F81022491C0800C0B2BF
S315080012E062689042CED3211D83B06846342200F04E
S315080012F0C5FD0EBC2068FFF730F8002804D0022090
S3150800130084F8BD0301200FE0002084F8380001208E
S3150800131084F8BD03606A012802D1200000F027FE88
S315080013202068FFF71EFE00200BB030BD10B5040084
S31508001330002C01D101200CE0032084F8BD03200015
S3150800134000F01EF8200000F026FE002084F8BD03F9
S31508001350002010BD10B5040094F8BC03012801D183
S3150800136002200CE0012084F8BC032068FFF7EBFD9F
S315080013702068FEF7CAFF002084F8BC03002010BDD1
S3150800138010B5040094F8BC03012801D1022016E028
S31508001390012084F8BC032068FEF7BDFF2068FFF72C
S315080013A088FD002804D0002084F8BC03012006E04C
S315080013B02068FFF7D6FD002084F8BC03002010BD86
S315080013C02DE9F041060035682F003068FFF713FE57
S315080013D0002840F077823068FFF7D1FD002800F03A
S315080013E071823068FFF7CBFD800705D53068406904
S315080013F010F00200316848613068FFF7C0FDC0068A
S315080014003FD53068806930F0100031688861D5F8BA
S31508001410208018F00F011C20414306EB010010F54F
S31508001420FE74C8F34340022816D147F6F07018EA4E
S31508001430000F20D0C8F30A1292B2E1682800FFF71D
S3150800144097FCE068C8F30A110844E060A169C8F38C
S315080014500A104118A1610EE0C8F3434006280AD1D4
S31508001460082216F571712800FFF782FCA169C8F3F6
S315080014700A104118A1613068806950F0100031687F
S3150800148088613068FFF77BFD000347D50025306883
S31508001490FFF77AFD04003FE0E0073BD52900C9B213
S315080014A03068FFF785FD80465FEAC87009D517EBF7
S315080014B0451010F53060012181602900300000F0E8
S315080014C00CFC5FEA087009D517EB451010F530607B
S315080014D0082181602900300000F0A2FC5FEAC8609C
S315080014E005D517EB451010F53060102181605FEACD
S315080014F0886005D517EB451010F53060202181600E
S315080015005FEA884006D517EB451010F530604FF4B2
S31508001510005181606D1C6408002CBDD13068FFF74E
S315080015202EFD400376D53068FFF738FD0400002508
S315080015306EE0E0076AD52900C9B23068FFF744FDB6
S3150800154080465FEAC87036D5012115F00F0011FAFA
S3150800155000F017F50061496B31EA000017F50061E4
S31508001560486317EB451010F510600121816030695A
S3150800157001281BD11C2000FB05F13144896C00FBB6
S3150800158005F23244526C114400FB05F23244916470
S31508001590002D0BD100FB05F03044006D002805D165
S315080015A016F5717201213068FFF73BFD2900C9B2B3
S315080015B0300000F008FD5FEA087005D517EB451006
S315080015C010F51060082181605FEAC86005D517EB41
S315080015D0451010F51060102181605FEA486005D556
S315080015E017EB451010F51060402181605FEA88709E
S315080015F005D517EB451010F51060022181605FEAEA
S31508001600086003D52900300000F0F3FA6D1C640861
S31508001610002C8ED13068FFF7B2FC00281CD517F5D0
S31508001620006040684008400017F50061486096F879
S31508001630F403012807D1002086F8F40300213000BE
S3150800164000F0A8FC02E0300000F008FD30684069B0
S3150800165010F00040316848613068FFF790FC0005DB
S315080016600DD517F500608068C00702D5300000F078
S31508001670DAFC3068406910F4006031684861306807
S31508001680FFF77DFC00011AD53068406910F000604C
S315080016903168486196F8F40300280DD1012086F8D0
S315080016A0F4033068406DC0F38300C6F8F8030121DF
S315080016B0300000F06FFC02E0300000F0B4FC306847
S315080016C0FFF75DFCC00440F1938017F500604068A1
S315080016D04008400017F50061486010213068FEF7A1
S315080016E040FF00203CE04FF67F3117EB401212F521
S315080016F01062916017EB401212F51062126832F40C
S31508001700001217EB401313F510631A6017EB40121B
S3150800171012F51062126852F0006217EB401313F5C7
S3150800172010631A6017EB401212F53062916017EBDE
S31508001730401111F53061096831F4001117EB4012B8
S3150800174012F53062116017EB401111F53061096826
S3150800175051F0006117EB401212F530621160401C1F
S3150800176071688842BFD317F50060C06950F0011050
S3150800177017F50061C861306B002812D017F50060B4
S31508001780D0F8840050F00B0017F50061C1F884000A
S3150800179017F50060406C50F00B0017F500614864BF
S315080017A011E017F50060406940F4005050F02B0036
S315080017B017F50061486117F50060006950F00B00E5
S315080017C017F50061086117F50060006830F4FE60DF
S315080017D017F50067386016F571723169C9B2306855
S315080017E0FFF71FFC3068406910F480503168486183
S315080017F03068FFF7C4FB800417D53068FFF7FFFB96
S315080018003068FEF7D8FEF06000F04CFD0100F26883
S31508001810D2B23068FEF710FD300000F0E8FB306801
S31508001820406910F40050316848613068FFF7A7FB3B
S31508001830000708D5300000F0D4FB3068406910F086
S315080018400800316848613068FFF799FBC0020AD57D
S315080018500021C9B2300000F011FC3068406910F46C
S315080018608010316848613068FFF789FB80020AD525
S315080018700021C9B2300000F0FAFB3068406910F464
S315080018800010316848613068FFF779FB400008D5D9
S31508001890300000F0FAFB3068406910F0804031688B
S315080018A048613068FFF76BFB40070BD53068446822
S315080018B0600702D5300000F0F2FB30684068044348
S315080018C030684460BDE8F08110B5040094F8BC03A4
S315080018D0012801D1022009E0012084F8BC03206810
S315080018E0FFF731FB002084F8BC03002010BD10B5BB
S315080018F0040094F8BC03012801D1022009E0012064
S3150800190084F8BC032068FFF72CFB002084F8BC038E
S31508001910002010BD10B5040094F8BC03012801D1BD
S3150800192002200CE0012084F8BC0384F83810C9B200
S315080019302068FFF7F3FA002084F8BC03002010BDE6
S3150800194070B5050000260800C0B200060CD50C00CC
S31508001950E4B214F00F041C20444305EB040010F114
S315080019603C04012060700BE00C00E4B214F00F0494
S315080019701C20444305EB040010F5FE74002060703B
S3150800198011F00F01217092B2A260E370607800280E
S3150800199001D02078E080DBB2022B01D10020207133
S315080019A095F8BC03012801D102200BE0012085F837
S315080019B0BC0321002868FEF710FE002085F8BC034A
S315080019C03000C0B270BD10B504000800C0B20006F1
S315080019D00BD50A00D2B212F00F021C20424304EBC8
S315080019E002003C30012242700BE00A00D2B212F02B
S315080019F00F021C20424304EB020010F5FE70002281
S31508001A00427011F00F01017094F8BC13012901D13D
S31508001A1002200AE0012184F8BC1301002068FEF7C1
S31508001A2039FE002084F8BC03002010BD38B51C0020
S31508001A300D00EDB215F00F051C235D4300EB050301
S31508001A4013F5FE73DA605C6100249C6100245C7007
S31508001A5011F00F041C700469012C00D11A6111F0F1
S31508001A600F0F06D10269D2B219000068FFF776F89F
S31508001A7005E00269D2B219000068FEF7A1FE00204F
S31508001A8032BDC9B211F00F011C2251430844D0F8E7
S31508001A901402704738B51C000D00EDB215F00F059D
S31508001AA01C235D4300EB05033C33DA605C610024CC
S31508001AB09C6101245C7011F00F041C700469012CF0
S31508001AC000D11A6111F00F0F06D10269D2B21900BE
S31508001AD00068FFF743F805E00269D2B2190000680A
S31508001AE0FEF76EFE002032BD38B504000D006068B2
S31508001AF02900C9B211F00F01884201D2012039E04C
S31508001B002800C0B200060CD52900C9B211F00F0191
S31508001B101C20414304EB010010F13C0101204870F0
S31508001B2009E02900C9B21C20414304EB010010F565
S31508001B30FE71002048700120887015F00F000870AB
S31508001B4094F8BC03012801D1022013E0012084F88F
S31508001B50BC032068FFF71EF915F00F0F06D114F520
S31508001B6071722169C9B22068FFF75BFA002084F810
S31508001B70BC03002032BD10B5040060680A00D2B26A
S31508001B8012F00F02904201D2012031E00800C0B2E3
S31508001B9000060BD50A00D2B212F00F021C204243EF
S31508001BA004EB02003C30012242700BE00A00D2B27C
S31508001BB012F00F021C20424304EB020010F5FE70DF
S31508001BC0002242700022827011F00F01017094F811
S31508001BD0BC13012901D102200AE0012184F8BC13B3
S31508001BE001002068FFF720F9002084F8BC030020D4
S31508001BF010BD2DE9FC4704000D00266837001C209F
S31508001C0000FB05F0204410F13C08D8F81400D8F879
S31508001C101810884201D201205DE0D8F81400D8F8DF
S31508001C201890B0EB0909D8F80800484501D2D8F849
S31508001C30089019F103095FEA990926E0D8F8140013
S31508001C40D8F818A0B0EB0A0AD8F80800504501D20F
S31508001C50D8F808A01AF103095FEA99092069C0B201
S31508001C60009053469BB22A00D2B2D8F80C10300026
S31508001C70FFF762F8D8F80C005044C8F80C00D8F8FA
S31508001C8018001AEB000AC8F818A017EB451010F54B
S31508001C901060806980B2484509D3D8F81800D8F88A
S31508001CA01410884203D2D8F814000028C6D1D8F8F0
S31508001CB01800D8F8141088420CD3012015F00F0527
S31508001CC010FA05F517F50060406B30EA050517F5BB
S31508001CD000677D630020BDE8F68738B505000C006F
S31508001CE029680800096C10EB441212F530629268F4
S31508001CF02B69012B62D113070ED55D4B9942C0F0B3
S31508001D008D80110440F18A8010EB441010F5306084
S31508001D104FF40041816081E0930606D510EB44102C
S31508001D2010F530602021816078E012F0280F75D117
S31508001D304F4B994209D3110407D510EB441010F5FF
S31508001D4030604FF40041816068E01C2101FB04F219
S31508001D502A44D2F8042210EB441010F530600069CA
S31508001D604003400B121A01FB04F02844C0F8142261
S31508001D7001FB04F02844D0F8080201FB04F22A44C7
S31508001D80D2F80422104401FB04F22A44C2F80802DD
S31508001D90002C0DD101FB04F105EB0100D0F810026F
S31508001DA0002805D115F5717201212868FFF739F960
S31508001DB02100C9B2280000F0F7F82FE02D4B994210
S31508001DC017D1110407D510EB441010F530604FF405
S31508001DD00041816022E0910605D510EB441010F50C
S31508001DE03060202181602100C9B2280000F0DCF8AB
S31508001DF014E0002C0DD11C2000FB04F02844D0F878
S31508001E001002002805D115F5717200212868FFF720
S31508001E1008F92100C9B2280000F0C6F8002032BD32
S31508001E2070B5040022681000156C10EB411212F50B
S31508001E30306292680E4EB54208D3120406D510EBEE
S31508001E40411010F530604FF400418160200000F029
S31508001E50A3F8B54208D32069012805D114F5717293
S31508001E6001212068FFF7DDF8002070BD00000000A2
S31508001E700B30544F0A31544F70470000103A07D3BD
S31508001E8030B4B1E83810103AA0E83810F9D230BCAE
S31508001E90530724BFB1E80810A0E8081044BF51F85A
S31508001EA0043B40F8043BD20724BF31F8022B20F844
S31508001EB0022B44BF0B7803707047121F17D35B00C1
S31508001EC009D151F8043B20F8023B1B0C121F20F8DD
S31508001ED0023BF6D20BE051F8043B00F8013B1B0A23
S31508001EE020F8023B1B0C121F00F8013BF3D238BF47
S31508001EF0121D521E24BF11F8013B00F8013BF8D809
S31508001F007047000070B403685B6A0C00E4B2002CEA
S31508001F1005D192B253EA0243006883621FE004685F
S31508001F20A46A13EB1443002409E005682600F6B2F8
S31508001F3005EB8605D5F8045113EB1543641C2500FB
S31508001F40EDB20E00F6B2761EB542EED30068C9B2FF
S31508001F5000EB810092B253EA0243C0F80031002038
S31508001F6070BC704789B200684162002070470168FA
S31508001F700122C0F8FC23002280F8F423886950F077
S31508001F8000608861486D40F0805050F00300486555
S31508001F90002070477047704780B510F57171D0F80A
S31508001FA0000400F0FEF901BD80B50B00DBB21C226F
S31508001FB0534300EB0302D2F80822C9B2D0F8000452
S31508001FC000F021FA01BD80B50B00DBB21C22534399
S31508001FD000EB0302926CC9B2D0F8000400F05EFA76
S31508001FE001BD80B5D0F8000400F013FB01BD38B57B
S31508001FF004000125E068002801D1002508E0E06812
S31508002000022801D1012503E09121464800F027FB6B
S315080020102900C9B2D4F8000400F0E5FAD4F800049F
S3150800202000F0B1FA31BD10B50400D4F8000400F090
S31508002030DDFA206810F56060006850F0010021683C
S3150800204011F560610860206A002804D036480168E6
S3150800205051F00601016000F02BFB10BD10B504001D
S3150800206000F027FBD4F8000400F0C9FA10BD80B5CB
S31508002070C9B2D0F8000400F0DEFA01BD80B5C9B2D5
S31508002080D0F8000400F0D5FA01BD10B5040001200F
S3150800209000F00DFBD4F8000400F0CFFA10BD10B51F
S315080020A00400002000F003FBD4F8000400F0C7FA8F
S315080020B010BD10B50178002931D11C4CC4F80004B4
S315080020C0C0F8C4425FF0A04020600620606002208D
S315080020D0E060002020610220A0610120E06100206C
S315080020E02062002060620020E06200202063200059
S315080020F0FFF75CF8002804D040F22511094800F0E3
S31508002100AEFA80212000FFF72DFF40220021200093
S31508002110FFF7F8FE802201212000FFF7F3FE0020DA
S3150800212010BD0000D45B000810ED00E0C0000020E0
S3150800213080B500210021D0F8C402FFF7F7F8C0B235
S3150800214000F09BF8C0B202BD80B500210021D0F88E
S31508002150C402FFF7FFF8C0B200F08FF8C0B202BDA4
S3150800216080B500210021D0F8C402FFF709F9C0B2F2
S3150800217000F083F8C0B202BD10B51C00002300238E
S315080021801300DBB2220092B2C9B2D0F8C402FFF73C
S31508002190D7FBC0B200F071F8C0B210BD80B50022FE
S315080021A00022C9B2D0F8C402FFF70DFCC0B200F095
S315080021B064F8C0B202BD80B500220022C9B2D0F8C8
S315080021C0C402FFF791FCC0B200F057F8C0B202BDD6
S315080021D080B500220022C9B2D0F8C402FFF7CBFCB2
S315080021E0C0B200F04AF8C0B202BDD0F8C422080056
S315080021F0C0B2000609D5C9B211F07F011C204143BF
S3150800220002EB010090F83E0008E0C9B211F07F0128
S315080022101C20414302EB010090F8FE01704780B58F
S3150800222000220022C9B2D0F8C402FFF773FBC0B27D
S3150800223000F023F8C0B202BD10B500240024C9B2CC
S31508002240D0F8C402FFF726FCC0B200F016F8C0B2F8
S3150800225010BD10B500240024C9B2D0F8C402FFF797
S31508002260E5FBC0B200F009F8C0B210BD80B5C9B22E
S31508002270D0F8C402FFF705FC02BD0021C0B2002851
S3150800228005D0022807D004D3032806D007E000208B
S3150800229006E0032004E0012002E0032000E003201A
S315080022A0C0B270470148006870470000040000206B
S315080022B080B5002801D1032018E0D0F8B832002BE9
S315080022C002D00023C0F8B832D0F8CC32002B02D0A6
S315080022D00023C0F8CC32002901D0C0F8B41201217D
S315080022E080F89C120270FFF7E4FEC0B202BD10B57A
S315080022F00400012084F89C02D4F8B802002806D00D
S315080023006168C9B22000D4F8B82252689047D4F858
S31508002310CC02002802D00020C4F8CC022000FFF727
S315080023201FFF0100C9B2002901D0C0B203E0200096
S31508002330FFF7FEFEC0B210BD1CB504000020ADF8C4
S315080023400000002901D1032009E0C4F8B812684644
S31508002350D4F8B812C96A8847C4F8CC02002016BD5A
S3150800236080B5FFF7F1FE02BD0020704780B5032255
S31508002370D0F8B832002B05D0C9B2D0F8B822126806
S31508002380904702001000C0B202BD80B5D0F8B8224E
S31508002390002A04D0C9B2D0F8B82252689047002063
S315080023A002BD10B5040004F2AA2000F035FD012094
S315080023B0C4F89402B4F8B002C4F8980294F8AA02D1
S315080023C010F01F00002803D002280DD006D311E014
S315080023D004F2AA21200000F075F912E004F2AA21FD
S315080023E0200000F0AEF90CE004F2AA21200000F06B
S315080023F0E0F906E094F8AA1211F080012000FFF730
S31508002400DAFEC0B210BD10B5040010000A00D2B240
S31508002410002A2CD114F5AA72D4F89412032912D1E1
S31508002420D1689368994210D29368D1685B1A936011
S315080024309168D368994201D2926800E0D268010097
S31508002440200000F052FD002010BDD4F8B802006943
S31508002450002808D094F89C02032804D12000D4F858
S31508002460B81209698847200000F047FDEBE7D4F861
S31508002470B802806900280FD094F89C0203280BD173
S31508002480C9B22000D4F8B822926990470100C9B2AF
S315080024900029D8D0C0B2D7E70320D5E710B5040085
S315080024A010000A00D2B2002A56D114F11402D4F848
S315080024B09412022944D1D168936899420FD293683D
S315080024C0D1685B1A936092680100200000F005FD50
S315080024D00023002200212000FFF7BBFE30E0D06871
S315080024E09168884217D15068D168884213D35068DA
S315080024F0D4F8981288420ED200220021200000F05B
S31508002500ECFC0020C4F898020023002200212000D9
S31508002510FFF79FFE14E0D4F8B802C068002808D078
S3150800252094F89C02032804D12000D4F8B812C9688C
S31508002530884780212000FFF73EFE200000F0E8FCD7
S3150800254094F8A002012805D12000FFF70DFF00200E
S3150800255084F8A002002010BDD4F8B802406900280B
S315080025600FD094F89C0203280BD1C9B22000D4F8E6
S31508002570B822526990470100C9B20029EAD0C0B210
S31508002580E9E70320E7E710B50400012084F89C0278
S315080025900020C4F89402002060600020C4F8A40259
S315080025A0D4F8BC02002806D06168C9B22000D4F865
S315080025B0B822526890474023002200212000FFF7E6
S315080025C0DBFD0120A4F864014020C4F86001402323
S315080025D0002280212000FFF7CFFD0120A0844020A3
S315080025E02062002010BD01740020704790F89C12EC
S315080025F080F89D12042180F89C120020704790F8FC
S315080026009C12042903D190F89D1280F89C12002090
S31508002610704780B590F89C12032908D1D0F8B812F3
S31508002620C969002903D0D0F8B812C96988470020BB
S3150800263002BD00207047002070470020704780B513
S31508002640012180F89C12D0F8B812002905D04168FB
S31508002650C9B2D0F8B82252689047002002BD80B5AA
S3150800266000F065FCFCE7000000690840884201D1DB
S31508002670012000E00020C0B2704780B54FF4005139
S315080026800548FFF7F1FF002801D0002002E000F01E
S315080026907AFC012002BD00000008024080B56420D3
S315080026A000F04FFC01BD80B500F04EFC01BD70473F
S315080026B07047704701000878491C097850EA0120DC
S315080026C080B2704710B500240A7812F06002002A1A
S315080026D009D0202A01D0402A2ED1D0F8B8229268F3
S315080026E0904704002AE04A78002A19D0012A1DD00A
S315080026F0032A18D0052A09D0062A04D0082A0CD09D
S31508002700092A06D015E000F07EF914E000F07EFAFA
S3150800271011E000F0AAFA04000DE000F023FB0AE03D
S3150800272000F03FFB07E000F05BFB04E000F062FB13
S3150800273001E000F089FB01E000F086FB2000C0B252
S3150800274010BD70B505000E000024307810F060004A
S31508002750002803D0202801D0402823D195F89C02D0
S31508002760401E022819D83079022811D231002800D3
S31508002770D5F8B822926890470400F08800280BD153
S315080027802000C0B2002807D1280000F0B6FB03E0FD
S315080027903100280000F058FB03E03100280000F063
S315080027A053FB03E03100280000F04EFB2000C0B2C6
S315080027B070BD70B505000E000024B188307810F0A1
S315080027C0600000280CD0202802D0402840F0148150
S315080027D031002800D5F8B8229268904704000FE126
S315080027E07078002872D001283AD0032840F0FF807C
S315080027F095F89C02022802D0032816D02BE0080080
S31508002800C0B200280CD00800C0B2802808D0C9B2CF
S315080028102800FFF7D0FC80212800FFF7CCFC03E056
S315080028203100280000F010FB19E0708800280ED14E
S315080028300800C0B200280AD00800C0B2802806D016
S31508002840F088002803D1C9B22800FFF7B4FC280095
S3150800285000F053FB03E03100280000F0F5FACAE067
S3150800286095F89C02022802D0032816D029E0080011
S31508002870C0B200280CD00800C0B2802808D0C9B25F
S315080028802800FFF798FC80212800FFF794FC03E056
S315080028903100280000F0D8FA17E0708800280FD118
S315080028A011F07F0F03D0C9B22800FFF791FC28006A
S315080028B000F023FB31002800D5F8B822926890472B
S315080028C003E03100280000F0BFFA94E095F89C0276
S315080028D0022802D003282BD084E00800C0B20028C2
S315080028E008D00800C0B2802804D03100280000F0C3
S315080028F0ABFA7BE00800C0B2000609D5C9B211F0F0
S315080029007F011420414305EB010010F1140108E092
S31508002910C9B211F07F011420414305EB010010F5FF
S31508002920AA71002008600222280000F0C9FA5DE0BA
S315080029300800C0B200060FD50A00D2B212F00F0284
S315080029401420424305EB0200808C002815D1310083
S31508002950280000F079FA49E00A00D2B212F00F0214
S315080029601420424305EB0200B0F86401002804D1A4
S315080029703100280000F068FA38E00800C0B2000606
S315080029800AD50A00D2B212F07F021420424305EBA0
S31508002990020010F1140609E00A00D2B212F07F0212
S315080029A01420424305EB020010F5AA760800C0B2CF
S315080029B0002803D00800C0B2802802D10020306069
S315080029C00AE0C9B22800FFF710FC002802D001204F
S315080029D0306001E00020306002223100280000F05B
S315080029E06FFA03E03100280000F02EFA03E0310008
S315080029F0280000F029FA03E03100280000F024FA44
S31508002A002000C0B270BDF8B505000E000020ADF874
S31508002A10000000270024708880B2000AC0B201288E
S31508002A200AD0022810D0032823D0062800F0A58053
S31508002A30072800F0B280C2E06946287CD5F8B4229F
S31508002A40126890470700BFE0287C002808D168462E
S31508002A50D5F8B812896A884707000220787007E017
S31508002A606846D5F8B812C96A884707000220787000
S31508002A70AAE0B078002808D002282CD018D3042859
S31508002A804FD03BD305285FD071E0D5F8B402406833
S31508002A90002807D06946287CD5F8B42252689047A2
S31508002AA0070004E03100280000F0CEF9641C63E05A
S31508002AB0D5F8B4028068002807D06946287CD5F87E
S31508002AC0B42292689047070004E03100280000F01D
S31508002AD0BBF9641C50E0D5F8B402C068002807D0DA
S31508002AE06946287CD5F8B422D2689047070004E0E6
S31508002AF03100280000F0A8F9641C3DE0D5F8B402BE
S31508002B000069002807D06946287CD5F8B4221269DE
S31508002B109047070004E03100280000F095F9641C8E
S31508002B202AE0D5F8B4024069002807D06946287C0F
S31508002B30D5F8B42252699047070004E0310028000E
S31508002B4000F082F9641C17E0D5F8B4028069002801
S31508002B5007D06946287CD5F8B422926990470700C1
S31508002B6004E03100280000F06FF9641C04E031002D
S31508002B70280000F069F9641C26E0287C002806D1A4
S31508002B806846D5F8B812496B8847070004E0310053
S31508002B90280000F059F9641C16E0287C002808D1A2
S31508002BA06846D5F8B812096B884707000720787079
S31508002BB004E03100280000F047F9641C04E0310005
S31508002BC0280000F041F9641CE4B2002C1DD1F088FD
S31508002BD0002817D0BDF8000000280ED0BDF8000068
S31508002BE0F188884202D3F088ADF80000BDF80020CD
S31508002BF03900280000F064F907E03100280000F0E9
S31508002C0023F902E0280000F078F9F1BD38B505008F
S31508002C108888002825D1C888002822D14888802895
S31508002C201FD28C7814F07F0495F89C02032803D1F0
S31508002C30280000F009F917E085F89E422100C9B27C
S31508002C402800FFF7ECFA280000F057F9E4B2002C48
S31508002C5003D0022085F89C0206E0012085F89C0234
S31508002C6002E0280000F0F0F831BDF8B505000E00C6
S31508002C7000243B4F708838703878022805D3310015
S31508002C80280000F0E1F8032068E095F89C02022885
S31508002C9002D003281ED056E03878002816D0387897
S31508002CA0686039782800FFF761FB04002000C0B28D
S31508002CB0002804D03100280000F0C6F809E02800F2
S31508002CC000F01BF9032085F89C0202E0280000F0BA
S31508002CD014F941E0387800280CD1022085F89C02C6
S31508002CE03878686039782800FFF74FFB280000F02D
S31508002CF004F927E038786968884220D06968C9B23B
S31508002D002800FFF742FB3878686039782800FFF713
S31508002D102DFB04002000C0B200280CD0310028008A
S31508002D2000F092F86968C9B22800FFF72EFB022066
S31508002D3085F89C0206E0280000F0DFF802E028008B
S31508002D4000F0DBF808E03100280000F07DF839785B
S31508002D502800FFF71AFB03242000C0B2F2BD0000CA
S31508002D604C10002080B5CA88012A02D000F06CF801
S31508002D7016E090F89C22521E012A02D9921E08D00B
S31508002D800CE000218160012210F1080100F098F89A
S31508002D9006E00122011D00F093F801E000F054F866
S31508002DA001BD80B590F89C22521E022A15D8CA8801
S31508002DB0022A02D000F048F811E00121C160D0F8DB
S31508002DC0A412002903D0C16851F00201C160022291
S31508002DD010F10C0100F074F801E000F035F801BDBF
S31508002DE080B54988012904D10121C0F8A41200F050
S31508002DF084F801BD80B590F89C22521E022A08D894
S31508002E004988012904D10021C0F8A41200F075F8F8
S31508002E1001E000F019F801BD38B504000878207003
S31508002E20481C01786170451C2800FFF743FC608048
S31508002E30681C451C2800FFF73DFCA080681C401C48
S31508002E40FFF738FCE08031BD10B504008021200072
S31508002E50FFF7B1F900212000FFF7ADF910BDF8B56D
S31508002E6004000D0017000026002C1ED0200000F0DC
S31508002E701DF84000801C388038783100C9B2685483
S31508002E80761C03203100C9B26854761C0AE0207803
S31508002E903100C9B26854641C761C00203100C9B2DE
S31508002EA06854761C20780028F1D1F1BD0200002074
S31508002EB001E0401C521C11780029FAD1C0B27047B3
S31508002EC080B513000222C0F894228361C3610A0008
S31508002ED00021FFF7B1F9002002BD80B513000A00F2
S31508002EE00021FFF7A9F9002002BD80B513000A00EA
S31508002EF00021FFF7AEF9002002BD80B50421C0F815
S31508002F009412002300220021FFF796F9002002BD43
S31508002F1080B50521C0F89412002300220021FFF78E
S31508002F2098F9002002BD80B5FFF7B8FB01BD80B552
S31508002F30FFF7B9FB01BD0000816170470904816193
S31508002F40704714490880704710B5FEF7FCF8124C14
S31508002F502168884216D311490878002806D101202D
S31508002F60087080210E48FFF7E7FF05E0002008708B
S31508002F7080210B48FFF7E2FFFEF7E5F805490988C7
S31508002F804018206010BD80B580210548FFF7D6FFA0
S31508002F9001BD00004410002030100020471000201A
S31508002FA00004024038B50400002C01D10120AEE02F
S31508002FB094F82000002802D1200000F0B0FA20681A
S31508002FC0006830F0020021680860FEF7CDF80500B9
S31508002FD02068406880070DD5FEF7C6F8401B0B2809
S31508002FE0F6D3606A50F400306062052084F8200049
S31508002FF001208CE02068006850F001002168086014
S31508003000FEF7B2F8050020684068C0070DD4FEF741
S31508003010ABF8401B0B28F6D3606A50F400306062A8
S31508003020052084F82000012071E0207E012806D1C1
S315080030302068006850F080002168086005E0206874
S31508003040006830F0800021680860607E012806D19B
S315080030502068006850F040002168086005E0206894
S31508003060006830F0400021680860A07E012806D17B
S315080030702068006850F020002168086005E0206894
S31508003080006830F0200021680860E07E012806D13B
S315080030902068006830F010002168086005E02068A4
S315080030A0006850F0100021680860207F012806D1CA
S315080030B02068006850F008002168086005E020686C
S315080030C0006830F0080021680860607F012806D192
S315080030D02068006850F004002168086005E0206850
S315080030E0006830F0040021680860A168E0680143C0
S315080030F020690143606901436068401E01432068F6
S31508003100C16100206062012084F82000002032BDE1
S3150800311030B4026890F820201300DBB2012B03D0EC
S31508003120D2B2022A40F07F80594AD2F8000250F003
S315080031300100C2F80002D2F8000230F47C50C2F84E
S315080031400002D2F800024B6A50EA0320C2F80002D5
S3150800315001200B7D13F01F0310FA03F3D2F81C02AB
S315080031609843C2F81C02C869002816D1D2F80C0286
S315080031709843C2F80C02486902EBC000CC684D6857
S31508003180C5EA0444C0F84042486902EBC0008C68AE
S315080031900D68C5EA0444C0F84442C869012816D136
S315080031A0D2F80C021843C2F80C02486902EBC000B8
S315080031B00C684D68C5EA0444C0F84042486902EB09
S315080031C0C0008C68CD68C5EA0444C0F844428869E2
S315080031D0002805D1D2F804029843C2F8040204E094
S315080031E0D2F804021843C2F804020869002805D177
S315080031F0D2F814029843C2F8140204E0D2F8140272
S315080032001843C2F81402086A012804D1D2F81C022D
S315080032100343C2F81C32D2F8000240084000C2F844
S315080032200002002004E0416A51F480214162012035
S3150800323030BC704738B5040094F82000012821D125
S31508003240022084F8200020680068400840002168B1
S315080032500860FDF789FF050020684068C0070DD59E
S31508003260FDF782FF401B0B28F6D3606A50F4003046
S315080032706062052084F82000012008E000206062D2
S31508003280002004E0606A50F400206062012032BD2C
S315080032900064004070B490F820500468A6688C68F2
S315080032A0002CFFD02C00E4B2012C02D0EDB2022D86
S315080032B06ED116F0E05F65D0C6F30164032C05D322
S315080032C0416A51F400014162012066E00125A540EA
S315080032D01D608B68002B09D10B68CD6855EA4355EC
S315080032E0036826013344C3F880510AE04B688D68A9
S315080032F055EAC305CB681D43036826013344C3F862
S3150800330080510B69056826013544C5F88431097D65
S3150800331001290BD1016823011944D1F8841151F40C
S315080033208071036825012B44C3F88411D1799379F8
S315080033301B0453EA0163517953EA012311790B43BC
S31508003340016825012944C1F88C31D17893781B048A
S3150800335053EA0163517853EA012311780B43016854
S3150800336022011144C1F88831016822011144D1F8BB
S31508003370801151F00101006822011044C0F8801143
S3150800338000200AE0416A51F400114162012004E07C
S31508003390416A51F480214162012070BC704710B423
S315080033A00200002092F820301C00E4B2012C02D062
S315080033B0DBB2022B07D11268926812EA8162B2EB7D
S315080033C0816F00D0012010BC704730B490F82040BF
S315080033D02500EDB2012D03D0E4B2022C40F098800E
S315080033E000290AD10468E46814F0030F10D1416A71
S315080033F051F40011416201208FE00468246914F039
S31508003400030F05D1416A51F400114162012084E09D
S3150800341004680D012C44D4F8B04114F004049460F7
S315080034209468002C07D104680D012C44D4F8B041E7
S31508003430640D146006E004680D012C44D4F8B0410C
S31508003440E408546004680D012C44D4F8B04114F023
S315080034500204D46004680D012C44D4F8B44114F075
S315080034600F04146104680D012C44D4F8B441C4F364
S315080034700724946104680D012C44D4F8B441240C43
S31508003480546102680C012244D2F8B8211A70026805
S315080034900C012244D2F8B821120A5A7002680C01AB
S315080034A02244D2F8B821120C9A7002680C01224400
S315080034B0D2F8B821120EDA7002680C012244D2F84A
S315080034C0BC211A7102680C012244D2F8BC21120AE6
S315080034D05A7102680C012244D2F8BC21120C9A7166
S315080034E002680C012244D2F8BC21120EDA710029B6
S315080034F006D10168C96851F020010068C16005E07D
S315080035000168096951F0200100680161002004E0A2
S31508003510416A51F480214162012030BC70477047EE
S31508003520DFF8DC04016851F0010101607047DFF83B
S31508003530D0040068400810F001007047DFF8C01496
S315080035400A6832F0F80252EAC0020A607047DFF8E9
S31508003550B4040068400810F001007047DFF8AC04B6
S31508003560006810F00C007047DFF8A004006810F03F
S31508003570F0007047DFF89404006810F4E0507047D4
S31508003580DFF88804006810F4604070470100DFF82F
S3150800359080040068084050EA014070470100DFF8DF
S315080035A070040068084050EA01407047DFF850048C
S315080035B00068400E10F001007047DFF858040068F4
S315080035C010F480007047DFF84C040068C0F38810D8
S315080035D07047DFF84004006810F440307047DFF8A1
S315080035E03404006810F03F007047DFF814040068E0
S315080035F0C00E10F001007047DFF804040068400FA1
S3150800360010F00100704780B5FFF78AFFFFF78FFFBC
S315080036100128FBD10020DFF8F4130860DFF8E01377
S3150800362008680090009ADFF8F803024000920098B4
S3150800363008601020FFF782FFFFF7B8FF0028FBD1CC
S31508003640FFF7D3FF0028FBD1FFF7D6FF0028FBD1F1
S31508003650DFF8D003DFF8BC130860DFF8CC03DFF827
S31508003660B8130860DFF8B4130860DFF8C003016810
S3150800367031F4FE410160016851F47F010160DFF811
S3150800368088030168490849000160016851F08071A2
S315080036900160002002BD10B5040000F05CF920604E
S315080036A0206800F06CF96060606800F073F9A0604B
S315080036B0606800F079F9E06010BD10B500240328B1
S315080036C024D1FFF763FFDFF86813401A04D0401EC1
S315080036D006D0401E0BD011E000F03DF904008DE045
S315080036E0FFF725FF002801D0DFF8484386E0FFF7FB
S315080036F02EFF002801D04FF400447FE000F02BF99C
S3150800370000F03DF900F050F9040077E00C2824D1C8
S31508003710FFF73CFFDFF82013401A04D0001F06D03D
S31508003720001F0BD011E000F016F9040066E0FFF761
S31508003730FEFE002801D0DFF8FC425FE0FFF707FF36
S31508003740002801D04FF4004458E000F004F900F0D6
S3150800375016F900F01FF9040050E0B0F5406F27D1C4
S31508003760FFF714FFDFF8D412884207D0DFF8D0122B
S31508003770884207D0B0F10C2F0BD011E000F0EBF81F
S3150800378004003BE0FFF7D3FE002801D0DFF8A4428F
S3150800379034E0FFF7DCFE002801D04FF400442DE0AA
S315080037A000F0D9F800F0EBF800F0FEF8040025E088
S315080037B0302823D1FFF7EAFEDFF88812401A04D032
S315080037C0103806D010380BD011E000F0C4F8040009
S315080037D014E0FFF7ACFE002801D0DFF858420DE0F0
S315080037E0FFF7B5FE002801D04FF4004406E000F0CC
S315080037F0B2F800F0C4F800F0CDF80400200010BDBF
S3150800380010B50024C02824D1FFF7C8FEDFF8381207
S31508003810401A04D0403806D040380BD011E000F0EA
S315080038209AF8040095E0FFF782FE002801D0DFF839
S3150800383004428EE0FFF78BFE002801D04FF40044C7
S3150800384087E000F088F800F09AF800F0A3F8040082
S315080038507FE0B0F5407F27D1FFF7A0FEDFF8EC1137
S31508003860884207D0DFF8E811884207D0B0F1032F65
S315080038700BD011E000F06FF804006AE0FFF757FE7E
S31508003880002801D0DFF8AC4163E0FFF760FE0028AE
S3150800389001D04FF400445CE000F05DF800F06FF8EA
S315080038A000F078F8040054E0B0F5405F27D1FFF740
S315080038B075FEDFF8A011884207D0DFF89C11884210
S315080038C007D0B0F1302F0BD011E000F044F8040017
S315080038D03FE0FFF72CFE002801D0DFF8584138E01A
S315080038E0FFF735FE002801D04FF4004431E000F020
S315080038F032F800F044F800F04DF8040029E0B0F57D
S31508003900404F26D1FFF74AFEDFF85011884207D00C
S31508003910DFF84C11884207D0B0F1C02F0BD011E068
S3150800392000F019F8040014E0FFF701FE002801D0A2
S31508003930DFF800410DE0FFF70AFE002801D04FF43A
S31508003940004406E000F007F800F019F800F022F845
S315080039500400200010BD80B50020FFF7FFFD0028F9
S3150800396004D0042804D0082804D006E0314805E02D
S315080039703C4803E000F022F800E02E4802BD10B5EE
S315080039800400FFF7F1FD3849C0F30310085CC44092
S31508003990200010BD10B50400FFF7ECFD3349800A7E
S315080039A0085CC440200010BD10B50400FFF7E8FD10
S315080039B02E49400B085CC440200010BD70B500209D
S315080039C00020FFF7FAFD002803D0B0F5800F02D0DB
S315080039D003E0184C02E0234C00E0164CFFF7FFFD0D
S315080039E00500FFF7F0FD0600B4FBF5F006FB00F650
S315080039F0FFF7EFFD000C401C4000B6FBF0F070BD71
S31508003A0000380240703802407438024008380240D4
S31508003A109038024004380240843802408838024010
S31508003A20FFFFF2EA10300024003000240C38024070
S31508003A30010003000024F40004000C000004000C3C
S31508003A400008000C100030004000C0000001000310
S31508003A50000200030010003000200030004000C0C3
S31508003A60008000C000127A00E45E0008205F0008AB
S31508003A7038B500F02AF9DFF804544021681C00F034
S31508003A803BF92870DFF8F8434021601C00F034F950
S31508003A9020702878FF2802D02078FF2804D18421B6
S31508003AA0DFF8E003FEF7DBFDDFF8DC430022DFF892
S31508003AB0DC132000FEF7FCFBDFF8D4132000FEF72A
S31508003AC03BFC0120FEF7F3FD2000FEF749FCD4F885
S31508003AD0C402FDF7F9FE00F00EFAB0F5FA6F03D24C
S31508003AE04FF4FA6000F004FA31BD10B5DFF89843D8
S31508003AF0D4F8C402FDF7FBFE2000FEF7F8FB002011
S31508003B00FEF7D5FD10BD70B505000C002000C0B24B
S31508003B10402804DBB921DFF86C03FEF7A0FD20007E
S31508003B20C0B200F069F8C0B2012804D0BD21DFF8A0
S31508003B305403FEF794FD00260EE0FFF7F8F930006F
S31508003B4080B2285C00F058F8C0B2012803D0C6211C
S31508003B50CC48FEF784FD761C30002100C9B280B23D
S31508003B6089B28842E9D370BD2DE9F04105000E00FF
S31508003B70C548D0F8C402FDF723FCC64C20780028B7
S31508003B8013D1C54D280000F02FF801280AD128784E
S31508003B90002807D02878402804DA01202070002061
S31508003BA0BE4908700020BDE8F081BC4FDFF8E88206
S31508003BB038784044401C00F017F80128F2D13878CC
S31508003BC0401C3870387898F800108842EAD13A785C
S31508003BD092B218F10101280000F0C6F90020207001
S31508003BE0387830700120DEE780B50100A4480078F7
S31508003BF000F0E7F8C0B202BD80B50100C9B29F481F
S31508003C00007800F090F8C0B202BD7CB59B4C2078D5
S31508003C1000F021F905002800C0B2002826D02800A7
S31508003C20C0B2412800DB4025002612E0694620780C
S31508003C3000F0C7F8C0B2012804D04FF4A371914828
S31508003C40FEF70DFD9DF8000095493200D2B2885462
S31508003C50761C30002900C0B2C9B28842E6D3EDB25C
S31508003C602B008F4A81218848FEF7E6FA73BDF8B51E
S31508003C700600002000F003FA0400834D3100C9B2A3
S31508003C802800FEF7F3FA070000260FE0300080B29E
S31508003C90215C7B48007800F046F8C0B2012804D0C1
S31508003CA04FF4B4717748FEF7DAFC761C3000390019
S31508003CB080B289B28842E9D300F0E1F902004023D4
S31508003CC001212800FEF7C5FAF1BD10B4754B19009D
S31508003CD013F11802002004E088744A61183118327A
S31508003CE0401C0400E4B2002CF6D088740020486119
S31508003CF06D48036010BC704710B46B4B1A68002AF5
S31508003D0001D1FF200DE01A6854691C601174906097
S31508003D10D060002353741060C9B20844401E506036
S31508003D20907C10BC704738B505000C002800C0B25E
S31508003D30022804DB4FF4E0715248FEF790FC182085
S31508003D4058492A00D2B242430A44527C2B00DBB2BD
S31508003D5043430B441B7C9A4201D1002030E02A00E1
S31508003D60D2B242430A44D26814702A00D2B24243FD
S31508003D700A442B00DBB243430B445B7C5B1C537445
S31508003D802A00D2B242430A442B00DBB243430B4417
S31508003D90DB685B1CD3602A00D2B242430A445268ED
S31508003DA02B00DBB243430B44DB689A4207D22A0056
S31508003DB0D2B242430A44EDB245434859D060012085
S31508003DC032BD38B504000D002000C0B2022804DB5D
S31508003DD04FF4F1712B48FEF742FC1821314A2000B6
S31508003DE0C0B248431044407C002801D1002031E08D
S31508003DF02000C0B24843104480680078287020002C
S31508003E00C0B2484310442300DBB24B4313445B7CE7
S31508003E105B1E43742000C0B2484310442300DBB243
S31508003E204B4313449B685B1C83602000C0B2484325
S31508003E30104440682300DBB24B4313449B68984206
S31508003E4007D22000C0B248431044E4B24C4311598B
S31508003E508160012032BD10B504002000C0B20228DE
S31508003E6004DB40F202210748FEF7F9FB0D49E4B2EC
S31508003E701820444301EB0400407C10BD2C0E0020A2
S31508003E80700E0020505D0008C40400206C0000205D
S31508003E90140000204B100020F40E00204A100020C9
S31508003EA0340F0020B40F00203C10002080B50120FC
S31508003EB01749087000F022F800F001F801BD10B5A6
S31508003EC000F078F9012812D0114C207801280ED17B
S31508003ED0FDF739F90F490A680F4909688A1812F572
S31508003EE0FA72904203D30020207000F01BF810BD30
S31508003EF008490860704707480068704780B5044855
S31508003F000078012803D1FDF71EF90349086001BDB1
S31508003F10461000202C1000202810002080B500F044
S31508003F2053F901BD10B500F05FF9002816D0FEF769
S31508003F30A4FB002812D000F0EBF8FDF7F7F800F024
S31508003F4070F900F055F9064908400649086000F07E
S31508003F504FF9001D046800F039F9A04710BD0000AC
S31508003F6080FFFF1F08ED00E070B504000D00160085
S31508003F7005E0287820706D1C641CFEF7D8FF300019
S31508003F80461E80B20028F4D170BD000038B5040082
S31508003F9000254023022281212000FEF7EDF8402368
S31508003FA0022201212000FEF7E7F84023354A0121C5
S31508003FB02000FEF74EF92800C0B232BD38B504001D
S31508003FC0002581212000FEF7E9F801212000FEF7EF
S31508003FD0E5F82800C0B232BD38B50B0017222A4CC6
S31508003FE014F109011D7815F0600F29D15D78062DA9
S31508003FF004D00A2D14D00B2D17D021E05D88ADB260
S315080040002D0AADB2212D07D114F11201DA88182A2A
S3150800401001DB172200E0DA8892B2FEF751FF0FE0C3
S3150800402001221A49FEF74CFF0AE05988C9B200294D
S3150800403003D198781549086002E01900FEF704FFD5
S31508004040002032BD80B5FFF7E0FD002002BD80B537
S315080040500800C0B2FFF70BFE002002BD80B590F83D
S315080040609C02032801D1FFF7D0FD002002BD2021C4
S315080040700180054870470A210180054870470148B4
S3150800408070470000740F00204C00002040100020EC
S315080040900800002010B500F0E9F800F035FB434CA5
S315080040A00120207000F015FC00202070FFF7E0FCCE
S315080040B00220207010BD1CB53D4C6946200000F05A
S315080040C0BBFB012807D10120384908709DF800106C
S315080040D0200000F0EBF86946200000F036FC0128C5
S315080040E007D10020314908709DF80010200000F023
S315080040F0DDF869462000FFF737FD012807D10220C1
S315080041002A4908709DF80010200000F0CFF813BD6A
S3150800411080B5FFF7EAFC01BD70B504000D00234E1B
S315080041203078012804D12900C9B2200000F055FBD7
S315080041303078002804D12900C9B2200000F0E4FB39
S315080041403078022804D12900C9B22000FFF7DBFC29
S3150800415000F0A6F870BD15480078002805D002289A
S3150800416007D004D3032806D007E0402006E008203D
S3150800417004E03F2002E0002000E0402080B27047C3
S315080041800A480078002805D0022807D004D3032857
S3150800419006D007E0402006E0082004E03F2002E0C1
S315080041A0002000E0402080B270470000BC000020DC
S315080041B0B40E002010B5002400F069F8002800D0DD
S315080041C001242000C0B210BD72B6704762B67047AF
S315080041D080B500F037FC01BD80B500F03CFC02BD9F
S315080041E080B500F06DFC02BD80B500F0C7FC02BDCD
S315080041F080B500F004FD02BD80B500F08AFC0028F9
S3150800420001D1002001E000F0E1FC02BD80B50320E9
S3150800421000F065FE002000F089FE00F0BBFF0020DC
S3150800422002BD80B50C485FF0FF31016000220260D4
S315080042300A48016000220260094801600022026003
S3150800424008480160002202600748016000210160F9
S3150800425001F012F8002002BD20380240243802403E
S31508004260103802401438024018380240DFF8C803F4
S315080042700021017000218164002180F8431000218B
S31508004280A0F8441000218170002141707047DFF8C2
S31508004290A8030078002801D1002000E0012070471B
S315080042A00020DFF8941381F84300704710B50178B1
S315080042B0FF2917D100F08CF8DFF87C4394F8430007
S315080042C0012802D1102000F07BF8B4F94400012837
S315080042D007DB012084F84300B4F94410E01C00F021
S315080042E053F810BDDFF85013097801294BD101782E
S315080042F0C92932D0CC293FD0CF293AD0D0292FD0BE
S31508004300D12933D0D2292ED0F32917D0F4290FD0AA
S31508004310F5290AD0F6290ED0FA2912D0FC2913D08D
S31508004320FD2914D0FE2915D029E000F0B5F8C3E719
S3150800433000F0D1F8C0E700F0A6F8BDE700F0ECF809
S31508004340BAE700F08EF8B7E700F086F8B4E700F0B1
S3150800435072F8B1E700F063F8AEE700F004F9ABE7EE
S3150800436000F020F9A8E700F0E9F8A5E700F048F919
S31508004370A2E700F057F99FE700F062F99CE72020D2
S3150800438000F01EF898E7ACE780B589B2FFF7C4FEDF
S3150800439001BDF8B504000D001600002704E02078DA
S315080043A0C719641CFEF7C3FD2800451E0028F6D170
S315080043B0FFB237600120F2BD00209F494870704760
S315080043C09D49FE22CA7008710220A1F84400704770
S315080043D010B5FFF7F1FF984C01202070FF20E07020
S315080043E000202071207950F01000207100206071A3
S315080043F060796071FFF7AFFEA071FFF7C1FEE0714B
S31508004400FFF7BEFE80B2000A20720120607201200A
S31508004410A0720820A4F84400FFF7DAFE10BD10B514
S31508004420854C00202070FFF7C7FFFF20E0700120B1
S31508004430A4F8440010BD8048FF21C1700021017115
S3150800444041784171002181710021C17100210172F9
S315080044500621A0F84410704780B50020FFF7B0FF8A
S3150800446001BD7548FF21C17074498164002101713D
S3150800447000214171002181710721C0F80710082128
S31508004480A0F8441070476C49FF22CA7040688864D7
S315080044900120A1F84400704738B50400FFF75BFE19
S315080044A080B2401E6178884203DA2220FFF788FF2F
S315080044B010E06278604D281D92B2A96CFFF754FD92
S315080044C0FF20E870A86C61784018A8646078401CE2
S315080044D0A5F8440031BD38B50400FFF73CFE80B2AC
S315080044E0401E6178884203DA2220FFF769FF12E04E
S315080044F0514D6068A8646278281D92B2A96CFFF7CE
S3150800450033FDFF20E870A86C61784018A8646078CD
S31508004510401CA5F8440031BD10B5474CFF21E17099
S31508004520E21D4168A06CFFF734FF2071002060711E
S315080045300020A0710820A4F8440010BD10B53E4C18
S31508004540FF20E0700020207100206071FFF703FE55
S31508004550A0710020E0710020207200206072072000
S31508004560A4F8440010BD38B50400FFF7F4FD0100B7
S31508004570314D621C89B2491EA86CFFF72DFE002832
S3150800458003D13120FFF71CFF0BE0FF20E870FFF78F
S31508004590E2FDA96C80B2401E4018A8640120A5F867
S315080045A0440031BD38B50400FFF7D5FD80B2801E42
S315080045B06178884203DA2220FFF702FF1FE01E4DCA
S315080045C0FF20E8700120A5F844006078002807D18C
S315080045D0FFF712FE002802D13120FFF7F1FE0EE0A8
S315080045E0A21C6178A86CFFF7F7FD002803D13120DB
S315080045F0FFF7E6FE03E0A86C61784018A86431BDB1
S3150800460010B50D4C4168A06CFFF7EAFD002803D1F0
S315080046103120FFF7D5FE04E0FF20E0700120A4F862
S31508004620440010BD80B5FFF77DFC0348FF21C1702B
S315080046300121A0F8441001BD9C0D0020305F000840
S3150800464080B53120FFF7BCFE01BD0000F8B584B087
S3150800465004000D0016001F006846FFF71CF80298B4
S315080046604FF47A71B0FBF1F1002200E0521C100001
S31508004670C0B2122845D2864B200080B294465FFA13
S315080046808CFC13F81CC096465FFA8EFE03EB4E0EA2
S315080046909EF801E01EEB0C0C1CF1010C0CFB00F063
S315080046A0B1FBF0FC00FB1C100028DFD1200080B213
S315080046B094465FFA8CFC13F81CC096465FFA8EFE89
S315080046C003EB4E0E9EF801E01EEB0C0C1CF1010CE0
S315080046D00CFB00F0B1FBF0F0288028880028C5D034
S315080046E0288840F2014C6045C0DA1000C0B213F8C1
S315080046F010003070D2B203EB4200407838700120C7
S3150800470000E0002005B0F0BD30B58BB00020ADF854
S31508004710020000208DF8010000208DF8000040F20C
S3150800472067656B460DF101020DF102014FF4FA704F
S31508004730FFF78CFF002803D1B5215648FDF78FFFF8
S31508004740554C5648206000202076002060760020D0
S31508004750A0760120E07600202077002060770020F0
S31508004760A0600020E0609DF80100401E0004206162
S315080047709DF80000401E00056061BDF802006060FB
S315080047802000FEF70FFC002D02D46D05444805E015
S3150800479025F00045ED0055F0040542480021069134
S315080047A000210791012108912900090C0191ADB258
S315080047B002950100090C039180B20490002005902F
S315080047C0012009900E200A9001A92000FEF7A0FCFE
S315080047D02000FEF72FFD0BB030BD30B587B00200C4
S315080047E040F2E170002803D401900020039004E011
S315080047F020F0004002900420039000200490C9B2E3
S315080048000591254D6B4601A92800FEF743FDC0B268
S3150800481000280FD1FCF797FC0400323400992800D1
S31508004820FEF7BDFD002805D0FEF781FBFCF78BFCE3
S315080048308442F3D207B030BD78B587B003000C00C8
S3150800484040F2676600256A4600211348FEF7BDFD5B
S31508004850002812D1002E07D40098B0420DD1029834
S3150800486000280AD1012508E026F000460198B04242
S3150800487003D10298042800D101252800C0B20128D6
S3150800488001D1049820702800C0B208B070BD00009D
S31508004890EC5D0008145D0008E40F00200064004089
S315080048A00400E0FFFCFF1F00016851F001010160F0
S315080048B07047C069400910F001007047C069C00917
S315080048C010F001007047406AC0B27047C9B28162F1
S315080048D0704718B587B04FF46140009000200190EA
S315080048E000200290002003900C20049000200590E0
S315080048F0002006904D4C6946200000F03CFD200043
S31508004900FFF7D2FF08B010BD70B504000D002800EF
S31508004910C0B2412803DB81214548FDF7A0FE2800E7
S31508004920C0B200F06BF8002607E0FEF700FB300087
S3150800493080B2205C00F062F8761C30002900C9B20B
S3150800494080B289B28842F0D370BD2DE9F0410500E6
S315080049500E00384C2078002815D1374D280000F075
S315080049603DF8012837D12878002834D028784128FE
S3150800497031DAFCF7E8FB3149086000203049087055
S315080049800120207027E02E4FDFF8AC8038784044AD
S31508004990401C00F023F8012814D13878401C3870E0
S315080049A0387898F80010884215D13A7892B218F1FA
S315080049B001012800FFF7D8FA0020207038783070F7
S315080049C0012009E0FCF7BFFB1C49096864318142F4
S315080049D001D2002020700020BDE8F08138B504001F
S315080049E0124D2800FFF765FF002805D02800FFF7BD
S315080049F06AFF2070012000E0002032BD38B50100B2
S31508004A000A4DC9B22800FFF761FFFCF79CFB0400BA
S31508004A100A342800FFF752FF002805D1FEF787FA67
S31508004A20FCF791FB8442F4D231BD000000480040F7
S31508004A30D45C000849100020E80D0020341000203E
S31508004A40481000205FF0FF30DFF8D4130860DFF865
S31508004A50D41308607047F8B504000D001600DFF897
S31508004A60C873B96CF86C4118491E091B681E814247
S31508004A7001D2002023E0200000F0A9F9FF2805D084
S31508004A802819401E00F0A3F9FF2801D1002016E0DE
S31508004A902100490A4FF4007041433868814207D122
S31508004AA02B0032002100DFF87C0300F0DCF806E07A
S31508004AB02B0032002100DFF8680300F0D4F8F2BDBD
S31508004AC070B504000D00DFF86003816CC06C4118F6
S31508004AD0491E091B681E814201D2002018E02000E9
S31508004AE000F075F906002C19641E200000F06FF915
S31508004AF03100C9B2FF2903D00100C9B2FF2901D18B
S31508004B00002005E00100C9B23000C0B200F01EF96D
S31508004B1070BD80B500200090C249086810F1010FE9
S31508004B2001D1012029E0009A486882180092009A6B
S31508004B30886882180092009AC86882180092009ABB
S31508004B40086982180092009A486982180092009AA9
S31508004B50886982180092009AC8698218009200989B
S31508004B60C04300900098401C00906A460421AE4855
S31508004B70006810F5E470FFF76EFF02BD0021AA4A2F
S31508004B801068006841181068001D00684118106810
S31508004B9008300068411810680C3000684118106821
S31508004BA01030006841181068143000684118106801
S31508004BB0183000684118106810F5E470006841184C
S31508004BC0002901D1012000E00020704780B59548F2
S31508004BD0016811F1010F05D000F08FF8002801D106
S31508004BE000200BE08E48016811F1010F05D000F096
S31508004BF084F8002801D1002000E0012002BD8A487F
S31508004C000068704780B5CA0501D000200BE002682D
S31508004C108A4201D1012006E001604FF40072001DAE
S31508004C20FFF7A2F9012002BD38B504000D007D4842
S31508004C30844208D17A4C29002000FFF7E3FF0028B8
S31508004C400FD100200EE078490A68954202D1040087
S31508004C500D68F0E7200000F050F80028EBD100209E
S31508004C6000E0200032BD2DE9F04104008846160018
S31508004C701D0047467F0A4FF400704743206810F12D
S31508004C80010F07D139002000FFF7BCFF002801D12A
S31508004C9000202EE02068B84208D039002000FFF72F
S31508004CA0C3FF0400002C01D1002022E02068B8EBE5
S31508004CB0000804EB080010F10408FEF738F9201D77
S31508004CC0B8EB0000B0F5007F09D317F50071200096
S31508004CD0FFF7AAFF0400002C0DD014F10408307861
S31508004CE088F8000018F10108761C6D1E002DE4D125
S31508004CF00120BDE8F0810020FBE72DE9F041050021
S31508004D00012600F001FC002704E0D8F80000A042C4
S31508004D1015D17F1C802F13D2D5F8008018EB870891
S31508004D2005EB87004468FEF702F922000023414696
S31508004D30022000F0A3FB0028E7D0002600E00026AA
S31508004D4000F0F2FB3000C0B2BDE8F08178B585B05E
S31508004D5004000D0001260020009028002100C0B2A2
S31508004D60C9B2884200D200262F482100027AC9B269
S31508004D70914205D390F850002900C9B2884200D262
S31508004D8000263000C0B201281DD100200190022063
S31508004D9004900120039000F0B7FB00E0641C280093
S31508004DA02100C0B2C9B288420BD3FEF7C0F8200072
S31508004DB0C0B20290694601A800F064FC0028EDD054
S31508004DC0002600F0B1FB3000C0B206B070BD70B569
S31508004DD00400FF25002600E0761C3000C0B2072834
S31508004DE01AD2FEF7A4F80C210F4A3000C0B2484385
S31508004DF010588442F0D33000C0B2484313583000EC
S31508004E00C0B2484310444068C3189C42E4D2F6B284
S31508004E104E4302EB0600057A2800C0B270BD0000BA
S31508004E2094070020980900202C5C000810F0070061
S31508004E30374B1A684FF6FF010A40364951EA0021F6
S31508004E400A431A60704732480068C0F30220704768
S31508004E50020052B2002A04D409012F4A40B2115462
S31508004E6007E009012D4A40B210F00F00104400F87F
S31508004E70041C704710B410F00700D0F10703052B87
S31508004E8001D3042301E0D0F10703041D072C01D246
S31508004E90002000E0C01E012414FA03F35B1E19402B
S31508004EA0814014FA00F0401E1040084310BC7047B9
S31508004EB080B5411EB1F1807F01D301200EE0401E6E
S31508004EC0174908600F215FF0FF30FFF7C1FF002088
S31508004ED014490860072014490860002002BD80B5FF
S31508004EE0FFF7A4FF01BD70B504000D0016000020F1
S31508004EF0FFF7A9FF32002900FFF7BCFF01002000D9
S31508004F0040B2FFF7A5FF70BD80B5FFF7D1FF02BD20
S31508004F100CED00E00000FA0500E400E018ED00E002
S31508004F2014E000E018E000E010E000E010B504002E
S31508004F304FF47A700D490978B0FBF1F00C4909680D
S31508004F40B1FBF0F0FFF7E0FF002801D001200CE0EC
S31508004F50102C09D2002221005FF0FF30FFF7C3FFB3
S31508004F6004480460002000E0012010BDBD000020B8
S31508004F700400002000000020D948016851F480315F
S31508004F8001607047D6490A6832F440421043086007
S31508004F907047D448016851F4802101607047D148B0
S31508004FA0016851F4803101607047CE480068400CB2
S31508004FB010F001007047CC490A6892089200104325
S31508004FC008607047C848006810F00C007047C6496A
S31508004FD00A6832F0F002104308607047C2490A684E
S31508004FE032F4E052104308607047BF490A6832F449
S31508004FF06042104308607047BA48016851F08071F2
S3150800500001607047B7480068400E10F0010070470D
S3150800501070B4B64D2E68B64C26403043084350EA65
S3150800502082101843286070BC704770B4AF4D2E6864
S31508005030B04C26403043084350EA82101843286093
S3150800504070BC704781B0AC490A6802430A600968B7
S3150800505008400090009801B07047A7490A6832EAEC
S3150800506000000860704781B0A4490A6802430A60D4
S31508005070096808400090009801B070479F490A687F
S3150800508032EA00000860704781B09D490A68024309
S315080050900A60096808400090009801B0704798496E
S315080050A00A6832EA00000860704781B095490A68C4
S315080050B002430A60096808400090009801B07047EA
S315080050C090490A6832EA0000086070478E490A6803
S315080050D0120912011043086070478B48006810F0E7
S315080050E00F00704709048161704780B500F005F824
S315080050F000F05CFB00F068FBFCE780B5FFF786F87C
S3150800510000F001F801BD80B50720FFF7DFFFFFF7C4
S31508005110E4FF072803D067217C48FDF7A0FA4FF47F
S315080051204040FFF72FFFFFF727FFFFF732FFFFF794
S3150800513036FFFFF73AFF0128FBD100234FF4D87258
S3150800514008215FF48000FFF763FF5FF010634FF4F8
S31508005150D87208215FF48000FFF767FFFFF74CFF5E
S31508005160FFF750FF0128FBD10020FFF730FF4FF46F
S31508005170A050FFF733FF4FF40040FFF736FF022039
S31508005180FFF719FFFFF71EFF0828FBD1604800F05C
S3150800519025FB01BD38B586B04FF48040FFF785FF83
S315080051A05FF08050FFF770FF0120FFF74BFF0220EA
S315080051B0FFF748FF0420FFF745FF0820FFF742FFE7
S315080051C05FF48020FFF760FF5FF00070FFF75CFF79
S315080051D0802000900120019000200290002003907A
S315080051E0002004904B4C6946200000F011FC8021F9
S315080051F02000FFF777FF4FF4005000900020019041
S31508005200002004906946444800F002FC4FF44075BB
S3150800521000950220019003200290002003900020B0
S3150800522004900720059069463C4800F0F1FB00957C
S315080052300220019003200290002003900020049091
S31508005240092005906946200000F0E2FB4FF4C050A3
S315080052500090022001900320029000200390002075
S3150800526004900A20059069462D4800F0D1FB80205D
S31508005270FFF7F9FE07B030BD10B5FEF7C4F9254CA7
S3150800528080212000FFF72EFF244800F02FFB22483C
S3150800529000F02CFB200000F029FB214800F026FB3B
S315080052A08020FFF7EBFE5FF00070FFF7F8FE5FF473
S315080052B08020FFF7F4FE0820FFF7CFFE0420FFF753
S315080052C0CCFE0220FFF7C9FE0120FFF7C6FE5FF0FD
S315080052D08050FFF7E4FE4FF48040FFF7F1FE10BD63
S315080052E00070004000380240083802400438024086
S315080052F00080BCFF0080BFF03038024034380240DE
S315080053004038024044380240003C0240805C0008B5
S3150800531000E6DF0C0004024000080240000C0240D0
S3150800532000000240006810F001007047426832F43D
S315080053304052114341607047826832F4407211430B
S3150800534081607047B2F5004F0ED11A00520812EB71
S315080053504102B2FBF3F189B24FF6F0720A40C1F38B
S3150800536042010A43C26005E011EB5301B1FBF3F1B8
S3150800537089B2C1607047F8B505000F000126002400
S315080053802800FFF7CFFF002862D129683A48014074
S3150800539078680143F868014338690143B8690143ED
S315080053A02960B9682800FFF7C1FF79692800FFF767
S315080053B0C3FF2948854204D10320FEF77EF904007D
S315080053C03AE02648854204D10C20FEF776F9040017
S315080053D032E02348854204D13020FEF76EF90400F6
S315080053E02AE02048854204D1C020FEF709FA0400C5
S315080053F022E01D48854205D14FF44070FEF700FAB9
S31508005400040019E01948854205D14FF44060FEF7BB
S3150800541054F9040010E01648854205D14FF440506F
S31508005420FEF7EEF9040007E01248854204D14FF46E
S315080054304040FEF7E5F90400002C09D0386800283A
S3150800544006D000263B68BA6921002800FFF77AFFD4
S315080054503000C0B2F2BD0000001001400044004018
S3150800546000480040004C0040005000400014014035
S3150800547000780040007C0040F369FFEF2DE9F8430F
S3150800548081460E0014001D000120DFF8E071387D0A
S31508005490012801D1022035E0012038754CF2503838
S315080054A0404600F048F80100C9B2002927D130006B
S315080054B022002B00B9F1000F07D0B9F1020F0ED068
S315080054C008D3B9F1030F0ED010E01100C9B200F0ED
S315080054D091F80BE0110089B200F07BF806E01100A4
S315080054E000F066F802E000F04EF8FFE7404600F0EC
S315080054F022F8DFF87C110A68520852000A60002177
S315080055003975C0B2BDE8F283002059490A68002AF5
S3150800551008D5594A594B1360594B13600968002935
S3150800552000D50120C0B270475148016851F00041CA
S3150800553001600020704738B50400002000204B4960
S315080055408861FBF711FE05004A480168C9030BD5B7
S3150800555014F1010FF8D0002C04D0FBF705FE401B10
S315080055608442F1D203200DE0016811F0F20F03D056
S3150800557000F04FF8012005E00168C90701D50121AF
S315080055800160002032BD10B439490C6834F4407407
S315080055900C600C6854F440740C600C6854F00104F8
S315080055A00C600260001D0360BFF34F8F10BC70478C
S315080055B02F4A136833F440731360136853F4007367
S315080055C01360136853F0010313600160BFF34F8F34
S315080055D07047274A136833F440731360136853F40B
S315080055E080731360136853F0010313600180BFF3DF
S315080055F04F8F70471E4A136833F44073136013685D
S315080056001360136853F0010313600170BFF34F8FE3
S31508005610704718480168890704D514498A6952F001
S3150800562020028A610168C90604D510498A6952F0C0
S3150800563010028A610168890604D50C498A6952F004
S3150800564008028A610168490604D508498A6952F040
S3150800565004028A610168090604D504498A6952F078
S3150800566002028A61F2210160704700000C100020D6
S31508005670103C02400C3C0240043C024023016745B2
S31508005680AB89EFCD2DE9F04104000D000120002083
S31508005690DFF81061307D012801D102203EE00120AB
S315080056A030754CF250373800FFF745FF0100C9B294
S315080056B0002930D15FF0FF312960216801290DD119
S315080056C0E068C0B200F02CF83800FFF734FFDFF8C6
S315080056D0D8100A6832F004020A601CE0D4F8048084
S315080056E001E018F10108A26861688A18904512D28B
S315080056F0E168C9B2404600F026F83800FFF71BFFFC
S3150800570029490A6832F07A020A600100C9B20029FA
S31508005710E7D0C5F8008000213175C0B2BDE8F08138
S3150800572021490A6832F440720A600A6852F0040293
S315080057300A600A68C0B2000250F48030104308605C
S31508005740BFF34F8F704700220A00D2B2002A01D158
S3150800575000210EE00A00D2B2012A02D14FF480716C
S3150800576007E0C9B2022902D14FF4007101E04FF4F3
S3150800577040710D4A136833F4407313601368194374
S315080057801160116831F0F80111601168C00050F01D
S31508005790020008431060106850F480301060BFF3B0
S315080057A04F8F70470C100020103C024080B5FEF762
S315080057B0B5FBFDF7B8FBFBF7A9FCFEF709FDFEF7FD
S315080057C069FCFEF773FB01BD80B5FDF7B0FBFBF77F
S315080057D0B1FCFEF770FCFEF772FB01BD01490860DB
S315080057E0704700000400002030B4046891FAA1F361
S315080057F0B3FA83F30325DBB25B009D40AC4391FA11
S31508005800A1F1B1FA81F1C9B249008A402243026086
S3150800581030BC704743688B43514319434160704716
S3150800582030B4846891FAA1F3B3FA83F30325DBB2A3
S315080058305B009D40AC4391FAA1F1B1FA81F1C9B27E
S3150800584049008A402243826030BC704730B4C4683D
S3150800585091FAA1F3B3FA83F30325DBB25B009D400B
S31508005860AC4391FAA1F1B1FA81F1C9B249008A4073
S315080058702243C26030BC704730B4046A91FAA1F37F
S31508005880B3FA83F30F25DBB29B009D40AC4391FA34
S31508005890A1F1B1FA81F1C9B289008A4022430262B4
S315080058A030BC704730B4446A0B001B0A93FAA3F362
S315080058B0B3FA83F30F25DBB29B009D40AC43090A7C
S315080058C091FAA1F1B1FA81F1C9B289008A4022435D
S315080058D0426230BC704742490A6810430860704704
S315080058E03F490A6832EA00000860704710B500248C
S315080058F03C49884206D10120FFF7EDFF0120FFF75A
S31508005900EFFF6AE03849884206D10220FFF7E3FF35
S315080059100220FFF7E5FF60E03449884206D10420FB
S31508005920FFF7D9FF0420FFF7DBFF56E0304988422E
S3150800593006D10820FFF7CFFF0820FFF7D1FF4CE07C
S315080059402C49884206D11020FFF7C5FF1020FFF723
S31508005950C7FF42E02849884206D12020FFF7BBFF4F
S315080059602020FFF7BDFF38E02449884206D14020B1
S31508005970FFF7B1FF4020FFF7B3FF2EE0204988422A
S3150800598006D18020FFF7A7FF8020FFF7A9FF24E0B4
S315080059901C49884208D14FF48070FFF79CFF4FF4EA
S315080059A08070FFF79DFF18E01749884208D14FF429
S315080059B00070FFF790FF4FF40070FFF791FF0CE0BF
S315080059C01249884208D14FF48060FFF784FF4FF4EC
S315080059D08060FFF785FF00E001242000C0B210BDFB
S315080059E0103802400000024000040240000802404D
S315080059F0000C024000100240001402400018024049
S31508005A00001C0240002002400024024000280240F8
S31508005A10F8B505000E0000200020306890FAA0F0C6
S31508005A20B0FA80F734E0726921002800FFF73AFFE0
S31508005A3028E034680120B8400440002C27D070685C
S31508005A40012802D07068022809D1B268210028000E
S31508005A50FFF7E6FEF26831682800FFF7DBFE3269D9
S31508005A6021002800FFF7F2FE706802280AD194FA8E
S31508005A70A4F0B0FA80F00828D5D27269210028006F
S31508005A80FFF7FAFE726821002800FFF7ADFE7F1CBB
S31508005A903068F8400028CCD10020F2BD12200880DA
S31508005AA02D487047042008802C48704780B50A00A6
S31508005AB0C0B2002804D12A492A48FDF7D0F903E0E4
S31508005AC027492848FDF7CBF9254802BD10B50A0035
S31508005AD0234C21002448FDF7C2F9200010BD80B5EB
S31508005AE01A20088000F022F8204802BD80B50A0076
S31508005AF0C0B2002804D11A491D48FDF7B0F903E0E1
S31508005B0017491B48FDF7ABF9154802BD80B50A00D1
S31508005B10C0B2002804D112491648FDF7A0F903E0DF
S31508005B200F491448FDF79BF90D4802BD38B51248D0
S31508005B30006812490C6812490968081800280AD032
S31508005B400A4D0822A91C00F01DF8042215F11201BD
S31508005B50200000F017F831BD880000209C000020C6
S31508005B609C0B0020D05E0008F45E0008A000002010
S31508005B70285F0008B85E000820F4F01F24F4F01F20
S31508005B8028F4F01F30B4002300231AE00400240F81
S31508005B9037341D00EDB201F815400AE00400240F61
S31508005BA00A2CF3D20400240F30341D00EDB201F89C
S31508005BB01540000100241D00EDB201EB45056C708F
S31508005BC05B1C1C001500E4B2EDB2AC42E6D330BC57
S31508005BD070470000433A5C576F726B5C736F66746C
S31508005BE0776172655C4F70656E424C545C546172A5
S31508005BF06765745C44656D6F5C41524D434D375F14
S31508005C0053544D333246375F4E75636C656F5F4646
S31508005C103734365A475F4941525C426F6F745C7538
S31508005C207362645F636F6E662E630000008000080F
S31508005C30008000000100000000000108008000004C
S31508005C400200000000800108008000000300000038
S31508005C50000002080000020004000000000004081A
S31508005C600000040005000000000008080000040009
S31508005C700600000000000C080000040007000000F1
S31508005C80433A5C576F726B5C736F667477617265C3
S31508005C905C4F70656E424C545C5461726765745C07
S31508005CA044656D6F5C41524D434D375F53544D33D8
S31508005CB03246375F4E75636C656F5F463734365AC2
S31508005CC0475F4941525C426F6F745C6D61696E2E25
S31508005CD063000000433A5C576F726B5C736F6674BF
S31508005CE0776172655C4F70656E424C545C546172A4
S31508005CF06765745C536F757263655C41524D434DBD
S31508005D00375F53544D333246375C72733233322E13
S31508005D1063000000433A5C576F726B5C736F66747E
S31508005D20776172655C4F70656E424C545C54617263
S31508005D306765745C536F757263655C41524D434D7C
S31508005D40375F53544D333246375C63616E2E6300BA
S31508005D50433A5C576F726B5C736F667477617265F2
S31508005D605C4F70656E424C545C5461726765745C36
S31508005D70536F757263655C41524D434D375F53549B
S31508005D804D333246375C7573622E630030B5016851
S31508005D9084684218416802EB5103C90703D54C448D
S31508005DA001E0491C05D19A420AD012F9011B12F8E2
S31508005DB0015B002904F8015BF3D4491EF7D5F2E725
S31508005DC00C3030BD10B5074979441831064C7C446F
S31508005DD0163404E00A68081D114488470146A142A2
S31508005DE0F8D110BD500000006C0000000502060244
S31508005DF0060307030803090309040A040B040C0431
S31508005E000C050D050E050F050F06100610071008E0
S31508005E104EF68851CEF20001086840F4700008601A
S31508005E20BFF34F8FBFF36F8F4FF00070E1EE100A8C
S31508005E30704700003FB3FFFF900F0000C00000202E
S31508005E400000000049FFFFFF940200003001000037
S31508005E500000002000F00DF8002801D0FFF7B2FF7F
S31508005E60AFF300800020AFF30080FFF73EF900F0A3
S31508005E7002F80120704700F001B8000007463846CE
S31508005E8000F002F8FBE7000080B5AFF30080024A95
S31508005E9011001820ABBEFBE7260002000448016883
S31508005EA051F4700101605FF00060024908607047B4
S31508005EB088ED00E008ED00E057696E555342204230
S31508005EC0756C6B20496E74657266616365000000C7
S31508005ED057696E5553422042756C6B204465766946
S31508005EE063650000000000000000000001020304D2
S31508005EF0060708094F70656E424C54205573657243
S31508005F000000000001488047014800479D5E0008E0
S31508005F10155F0008AFF30080FFF77AFFFFF79AFFD7
S31508005F20000000000102030444656661756C740094
S31508005F304F70656E424C5400FFF7FEBFFFF7FEBF79
S31508005F40FFF7FEBFFFF7FEBFFFF7FEBFFFF7FEBF77
S31508005F50FFF7FEBFFFF7FEBFFFF7FEBFFFF7FEBF67
S31508005F60FFF7FEBFFFF7FEBFFFF7FEBFFFF7FEBF57
S31508005F70FFF7FEBFFFF7FEBFFFF7FEBFFFF7FEBF47
S31508005F80FFF7FEBFFFF7FEBFFFF7FEBFFFF7FEBF37
S31508005F90FFF7FEBFFFF7FEBFFFF7FEBFFFF7FEBF27
S31508005FA0FFF7FEBFFFF7FEBFFFF7FEBFFFF7FEBF17
S31508005FB0FFF7FEBFFFF7FEBFFFF7FEBFFFF7FEBF07
S31508005FC0FFF7FEBFFFF7FEBFFFF7FEBFFFF7FEBFF7
S31508005FD0FFF7FEBFFFF7FEBFFFF7FEBFFFF7FEBFE7
S31508005FE0FFF7FEBFFFF7FEBFFFF7FEBFFFF7FEBFD7
S31508005FF0FFF7FEBFFFF7FEBFFFF7FEBFFFF7FEBFC7
S31508006000FFF7FEBFFFF7FEBFFFF7FEBFFFF7FEBFB6
S31508006010FFF7FEBFFFF7FEBFFFF7FEBFFFF7FEBFA6
S31508006020FFF7FEBFFFF7FEBFFFF7FEBFFFF7FEBF96
S31508006030FFF7FEBFFFF7FEBFFFF7FEBFFFF7FEBF86
S31508006040FFF7FEBFFFF7FEBFFFF7FEBFFFF7FEBF76
S31508006050FFF7FEBFFFF7FEBFFFF7FEBFFFF7FEBF66
S31508006060FFF7FEBFFFF7FEBFFFF7FEBFFFF7FEBF56
S31508006070FFF7FEBFFFF7FEBFFFF7FEBFFFF7FEBF46
S31508006080FFF7FEBFFFF7FEBFFFF7FEBFFFF7FEBF36
S31508006090FFF7FEBFFFF7FEBFFFF7FEBFFFF7FEBF26
S315080060A0FFF7FEBFFFF7FEBFFFF7FEBFFFF7FEBF16
S315080060B0FFF7FEBFFFF7FEBFFFF7FEBFFFF7FEBF06
S315080060C0FFF7FEBFFFF7FEBFFFF7FEBFFFF7FEBFF6
S315080060D0FFF7FEBFFFF7FEBFFFF7FEBF0010FC008D
S315080060E00624F4000A060002FD00014001FD000B2B
S315080060F08D3F0008BD3F0008D93F0008F8000B4552
S315080061004000084F4000085D400008F400036F4057
S315080061100008FC001277400008090220000101006F
S31508006120C0320904000002FFFD002D070581024068
S3150800613000FF070501024000FF9D5A0008A55A0006
S3150800614008CD5A0008AD5A0008DF5A0008ED5A0073
S31508006150080D5B000812010002FD001240501DAC3C
S31508006160600002010203010000040309041A03E6A1
S309080061700001040117
S70508005F157E
